:1000000000308A00BA290000FF00030E8301A1001E
:100010007F08A0000A08A8008A01A00E0408A20018
:100020007708A3007808A4007908A5007A08A6003C
:100030007B08A700831383128C308400801D222844
:100040008C193528220884002308F7002408F800BA
:100050002508F9002608FA002708FB0028088A006E
:10006000210E8300FF0E7F0E09008A1143280A101B
:100070008A100A118207023406340E341E343E34CC
:100080007E34FE34FF34680893008C118A112228D4
:100090006F308400000803195D280130F800BF307C
:1000A000F7006400F70B5128F80B4F284230F70097
:1000B000F70B58286400800B4D2800348316051771
:1000C0008312051F65280513662805178316051377
:1000D00083128A115A2AEF016F08F93C031C8B28FE
:1000E0006E1874280513752805178316051301303B
:1000F0008312EE066E187E2885137F2885178316D7
:10010000851364001F30F700F70B842800000000FF
:100110008312EF0A6C2883160513831205178316C2
:100120008513831285178A11A32A69088400700831
:100130008000840A8001E90A00347108F801700225
:100140000318A5287008F700B128F7010830F2005D
:10015000F00DF70D710877020318F700F80DF20B98
:10016000A828003478086E08F0006430F1009D2063
:100170007708EE0078083030031DC528EF1CCC2826
:10018000EF19CC286F1A2030C828EF116F126F14A6
:10019000F8077808F00095206E08F0000A30F100AA
:1001A0009D207708EE0078083030031DDD28EF1918
:1001B000E1286F1CE1286F1A2030F8077808F0005A
:1001C00095203030EE076E08F00095200034BC0119
:1001D000391CEC283910ED2839140034391C1A293F
:1001E000831686128312861264004730F700F70BDD
:1001F000F7280000831686128312861664004730A3
:10020000F700F70B0129000083168612831286126D
:1002100064004730F700F70B0B29000083168612A5
:100220008312861664001830F700F70B15290000BA
:1002300000002D29831686128312861264008530F1
:10024000F700F70B212983168612831286166400A5
:100250006F30F700F70B2A2900000034F101710814
:10026000073C031C762970080139F200BE08031907
:100270003B2900303C290130F300BD080319422915
:100280000030432901307305003A031956297208DA
:10029000F3000310BB0CBA0C030801397306013CD0
:1002A000031D56298430BB060830BA06F208031D28
:1002B0005B29E7207129BD080319BC0ABD08031991
:1002C0006329003064290130F3003C08053C031920
:1002D0006B2900306C290130730503197129EE2058
:1002E000E720EE200310F00CF10A2F29003439101A
:1002F000FF30BB00BA00BC010130BD00BE01BF0130
:100300003F08093C031C89297E30F0002E21BF0ADA
:100310008029BD01BF013F080F3C031C98292930EB
:100320003F0784000008EF00F0002E21BF0A8B2950
:10033000BF016E08840000080319A7296E08840015
:100340000008EF00F0002E21EE0ABF0A99290130C3
:10035000BE00FF30BA06BB063A08F0002E213B086B
:10036000F0002E21BE010130BD007E30F0002E21B4
:100370008A110C2B84011F30830583161F129F12D4
:100380001B0880399B0007309C0082308312A90033
:100390009830AA00AB004030AC00AD00AE00603039
:1003A000AF008630B000B430B1006030B200A4308D
:1003B000B300B400B5006130B6000330B700F030D0
:1003C000B800E90183160108C03981000E30F7003A
:1003D000073083128101813084000008F03907382A
:1003E000800064000008F739F719F03977048000BD
:1003F000900183161F129F121B088039D3389B006F
:100400001F1383121F179F1783169F1383121F1426
:10041000941283160611861406120030831294007B
:100420008316940007309C00050864000230F70032
:10043000F70B182A00001C0883120D1383169D0168
:1004400086118312861183160611831206118316F4
:1004500086108312861083168513831285178316E0
:100460000513831205172030F8001F08C7397804D8
:100470009F00950183168611831286110C30970018
:100480000030F80004389200643083169200623025
:100490008F00023083129500EA01831686108312C2
:1004A00086106430EF0048206A08EA0A043C031D05
:1004B0005B2A5E28EA0183168610831286140130B7
:1004C000EF0048201F151F19632A1E085F3C031CFC
:1004D0004D2A83168610831286100030F8001F08FC
:1004E000C73978049F0064001F30F700F70B762AA5
:1004F000000000001F151F197B2A1E08F7000310BB
:10050000F70C7708283EEB000830F8001F08C739C1
:1005100078049F0064001F30F700F70B8D2A00005D
:1005200000001F151F19922A03101E0CEC009501E4
:100530000030F800043892006B08831692001330E4
:10054000831295006B280230EE00FA30EF0048204D
:10055000EE0BA52A83168610831286142030F8002D
:100560001F08C73978049F0064000F30F700F70BAD
:10057000B72A00000130EA006A080A3C031CDC2AA2
:100580001F151F19C12A1E08ED006D08693C0318CC
:10059000CB2AEB0ACC2AEB0395010030F800043893
:1005A00092006B088316920013308312950064301A
:1005B000EF004820EA0ABC2A8316861083128610B0
:1005C0004030E9007030F00095203D30F00095207B
:1005D0006B08EE001B30EF00B2202030F0009520B9
:1005E0007230F00095203D30F00095206C08EE0050
:1005F0001B30EF00B2202030F00095207530F00065
:1006000095203D30F00095206D08EE001B30EF0086
:10061000B2204030EE0077293430EE00FA30EF009F
:100620004820EE0B0E2B8316940122308312940087
:100630000230E80068089300C0308B0483168C15E4
:100640008312EA016A08073C031C2F2B6A08372033
:10065000F800E8006C08EF004820EA0A222B831615
:1006600094018312940183168C11061183120615CE
:100670000A30EE008230EF004820EE0B3A2B831652
:0A068000061183120611432B6300DC
:04400E003C27FC3F10
:00000001FF
